:10000000830102308A00A42AFC0003088301D8007F
:100010000408D9000A08DA008A017008EA007108A9
:10002000E1007208E0007308E7007408E800750852
:10003000DF007608EB007708EC007808E20079082A
:10004000E9007A08E6007B08E5006308E4005B0845
:10005000DD005C08DE0083120B1C432A0317060830
:10006000B8003706B90097080319391EE228DF01E6
:10007000151C3C281030DF00BA0111083A020318A1
:100080007F281308BB00060810395F06031D53289C
:10009000BB0B4B283F2A000000004328BB0B512814
:1000A0003F2A00000000060810395F06031D4E2895
:1000B000951A60283A08433E84008317060874287E
:1000C0000608BC000608BD000608BE003A08433E0C
:1000D000840083173C083E05F0003D083E05F10012
:1000E0003C083D05710470048000151D7C280A162B
:1000F0008A112C250A128A110317BA0A3D28951C69
:10010000A3281408BB00060810395F06031D9328B6
:10011000BB0B8B283F2A000000008328BB0B9128D3
:100120003F2A00000000060810395F0603199E28C8
:100130008E28BB0B9C283F2A0000000006081039BF
:100140005F060319992899019A019B019C01C31C20
:100150001914C41C9914C51C1915C61C9915C71C63
:100160001916C81C9916C91C1917CA1C9917CB1C3B
:100170001A14CC1C9A14CD1C1A15CE1C9A15CF1C1F
:100180001A16D01C9A16D11C1A17D21C9A17D31CF7
:100190001B14D41C9B14D51C1B15D61C9B15D71CDB
:1001A0001B16D81C9B16D91C1B17DA1C9B17DB1CB3
:1001B0001C14DC1C9C14DD1C1C15DE1C9C159701FA
:1001C000970A3F2AA4080319B91E9129DF01221CAE
:1001D000EB282030DF00BA011E083A0203182E294E
:1001E0002008BB00060820395F06031D0229BB0B4F
:1001F000FA283F2A00000000F228BB0B00293F2A02
:1002000000000000060820395F06031DFD28A21A21
:100210000F293A08433E840083170608232906085D
:10022000BC000608BD000608BE003A08433E840034
:1002300083173C083E05F0003D083E05F1003C08F0
:100240003D05710470048000221D2B290A168A11B5
:100250002C250A128A110317BA0AEC28A21C52296B
:100260002108BB00060820395F06031D4229BB0B8D
:100270003A293F2A000000003229BB0B40293F2ABF
:1002800000000000060820395F0603194D293D29AA
:10029000BB0B4B293F2A00000000060820395F06EF
:1002A00003194829A601A701A801A901431D261485
:1002B000441DA614451D2615461DA615471D2616C8
:1002C000481DA616491D26174A1DA6174B1D2714A3
:1002D0004C1DA7144D1D27154E1DA7154F1D271684
:1002E000501DA716511D2717521DA717531D28145F
:1002F000541DA814551D2815561DA815571D281640
:10030000581DA816591D28175A1DA8175B1D29141A
:100310005C1DA9145D1D29155E1DA915A401A40A63
:100320003F2AB1080319391F3F2ADF012F1C9A29E0
:100330004030DF00BA012B083A020318DD292D08EE
:10034000BB00060840395F06031DB129BB0BA92974
:100350003F2A00000000A129BB0BAF293F2A000063
:100360000000060840395F06031DAC29AF1ABE29FC
:100370003A08433E840083170608D2290608BC00C9
:100380000608BD000608BE003A08433E84008317F5
:100390003C083E05F0003D083E05F1003C083D05E7
:1003A0007104700480002F1DDA290A168A112C2589
:1003B0000A128A110317BA0A9B29AF1C012A2E08B8
:1003C000BB00060840395F06031DF129BB0BE92974
:1003D0003F2A00000000E129BB0BEF293F2A000063
:1003E0000000060840395F060319FC29EC29BB0B05
:1003F000FA293F2A00000000060840395F06031969
:10040000F729B301B401B501B601C31D3314C41DEE
:10041000B314C51D3315C61DB315C71D3316C81D2E
:10042000B316C91D3317CA1DB317CB1D3414CC1D09
:10043000B414CD1D3415CE1DB415CF1D3416D01DEA
:10044000B416D11D3417D21DB417D31D3514D41DC5
:10045000B514D51D3515D61DB515D71D3516D81DA6
:10046000B516D91D3517DA1DB517DB1D3614DC1D81
:10047000B614DD1D3615DE1DB615B101B10A06082C
:10048000B7000B10831203130C1D672A8316201567
:100490003B08BF003C08C0003D08C1003E08C20048
:1004A000831215088316BB00831216088316BC003E
:1004B0003908BD003A08BE0083120C1C662A831658
:1004C000BC1B652ABD0A0319BE0A83120C110A1649
:1004D0008A112C250A128A118316201F7B2A0730C5
:1004E000C9000A168A15E9240A168A1526260A1250
:1004F0008A1183162013031383126A08F00061081F
:10050000F1006008F2006708F3006808F4005F0873
:10051000F5006B08F6006C08F7006208F80069083F
:10052000F9006608FA006508FB006408E3005D084E
:10053000DB005E08DC00590884005A088A0058086D
:100540008300FC0E7C0E0900203084005830BD2250
:10055000A0308400CB30BD2210308400603083177F
:10056000BD2290308400F0308317BD2283010A162B
:100570008A118C2904068001840A040603190034B8
:10058000BA2ADB00DC1BCD2A5C1BD52A5C088A005A
:100590005B08DB0A0319DC0A820083135C188317EB
:1005A0005B08DB0A840000080800831203135C0C5C
:1005B0001F3903178F0003135B0C03178D0083167D
:1005C0008C170C140000000083120C0803135B1836
:1005D000F02A031703108C1B03140E0D8312031350
:1005E0007F3908006C346134743468346534003405
:1005F000723435342034623431340034643472342B
:100600006F343334353430340034F5306136793971
:100610006F00F0392036803C34196931003AE539F1
:100620006536F43169007437EE328039683A003942
:100630006F3820366F386E008037693220396F335B
:100640006F000037F3376C386E107400EF370036E8
:10065000F5306F3A66336400F234721080326F38CE
:100660002036653763003100B9163000B9166200D4
:10067000E431801B693136376F006633A0390019C9
:10068000E637733331100000733465346C346534ED
:1006900063347434003464346934613400340A12CD
:1006A0008A15A52F0A168A15352C0A128A15F42DDB
:1006B0000A128A15CF2D0A128A15782D0A168A1564
:1006C000672C0A128A15682E0A128A15732F0A12CD
:1006D0008A152B2E0A168A15472C0A128A15472FBF
:1006E20083120313CF1F762B772B8B2B4C08F00032
:1006F2004D08F1004E08F2004F08F300F009F1092D
:10070200F209F309F00A0319F10A0319F20A0319AB
:10071200F30A962B831203134C08F0004D08F100E4
:100722004E08F2004F08F300962B031383120800C1
:100732009B2B6400831603178C189A2B031336081D
:10074200831203178D0083160313370883120317CE
:100752008C0083168C1303108B1B03148B130C1544
:1007620055308D00AA308D008C140C1103188B1794
:10077200031383120800831603132E08B70099236C
:100782008316B60A2F08B700992B831603132E0877
:10079200B70099238316B60A2F08B7009923831648
:1007A200B60A3008B70099238316B60A3108B70093
:1007B200992B831203133A08073A031D08005F2E90
:1007C20003172818EA2B3A3083120313C10046306C
:1007D200EF2B573083120313C1004630C200903012
:1007E2000A168A1546270A128A1183160317481811
:0E07F200002C3A3083120313C1004630052C50
:10080000573083120313C1004630C200B0300A16BD
:100810008A1546270A128A11831603176818162CA0
:100820003A3083120313C1004630682D57308312CB
:100830000313C1004630682D0317A818252C30304B
:1008400083120313C10046302A2C5E308312031337
:10085000C1004630C20090300A168A1546270A1297
:100860008A1183160317C8183B2C303083120313E8
:10087000C1004630402C5E3083120313C100463065
:10088000C200B0300A168A1546270A128A1183164A
:100890000317E818512C303083120313C10046307F
:1008A000682D5E3083120313C1004630682D831219
:1008B00003171008023A031D622C6F300313C100A6
:1008C00046306D2C100B692C74300313C100463078
:1008D0006D2C18300313C1004630C20090300A1648
:1008E0008A1546270A128A1103171D08023A031DAA
:1008F0007E2C6F300313C1004630892C1D0B852CD4
:1009000074300313C1004630892C18300313C10022
:100910004630C200B0300A168A1546270A128A11DC
:1009200003172A08023A031D9A2C6F300313C100E3
:100930004630682D2A0BA12C74300313C1004630B9
:10094000682D18300313C1004630682D65308312BE
:10095000C1004630C20090300A168A1546270A3078
:10096000F200F301831603172608F1002508F000B2
:100970000A168A15FE24740883120313C100750831
:10098000C20090300A168A1568266530C1004630CC
:10099000C200B0300A168A1546270A30F200F30169
:1009A000831603174608F1004508F0000A168A1559
:1009B000FE24740883120313C1007508C200B0300E
:1009C0000A168A1568266530C1004630C200D0304C
:1009D0000A168A1546270A30F200F3018316031718
:1009E0006608F1006508F0000A168A15FE240A124E
:1009F0008A11740883120313C1007508C200382DD0
:100A00002C308312C1004630C20090300A168A157D
:100A1000462783160317270883120313C100C20158
:100A200090300A168A1568262C30C1004630C20064
:100A3000B0300A168A154627831603174708831213
:100A40000313C100C201B0300A168A1568262C3083
:100A5000C1004630C200D0300A168A1546270A1255
:100A60008A1183160317670883120313C100C2019A
:100A7000D030D02D83120317951A432D4430031321
:100A8000C1004630472D11300313C1004630C2006B
:100A900090300A168A1546270A128A110317A21ADD
:100AA000562D44300313C10046305A2D1130031324
:100AB000C1004630C200B0300A168A1546270A1215
:100AC0008A110317AF1A6B2D44300313C10046304F
:100AD000C200D030C52D11300313C1004630682D3F
:100AE00025308312C1004630C20090300A168A15A4
:100AF0004627B0300A168A15D42483164708831275
:100B0000C100C201B0300A168A1568260A128A117D
:100B1000A52D0A308312C1004630C20090300A165B
:100B20008A1546270A128A118316211C9C2D4130F2
:100B30008312C1004630A02D53308312C1004630CD
:100B4000C200B0300A168A154627D0300A168A1518
:100B5000D4240A128A11812E50308312C1004630EB
:100B6000C20090300A168A154627B0300A168A1538
:100B7000D4240A128A118316AD08031DCB2D3730F9
:100B80008312C1004630C200B0300A168A154627CB
:100B90000A128A11812E2D088312C100C201B030C1
:100BA0000A168A1568260A128A11812EB601853026
:100BB000B70099238316B601B60A03172708031353
:100BC000B700992302308316B600031747080313B2
:100BD000B700992303308316B60003176708031381
:100BE000B7009923903083260A128A11B0308326E9
:100BF0000A128A11D03083260A128A11073083160E
:100C0000B60083120317100883160313B700992345
:100C100008308316B600831203171D0883160313CA
:100C2000B700992309308316B600831203172A08E8
:100C300083160313B700992383160317250803139C
:100C4000AE00031726080313AF000A30B600BC231A
:100C50000A128A118316031745080313AE000317FF
:100C600046080313AF000C30B600BC230A128A11E9
:100C70008316031765080313AE00031766080313F2
:100C8000AF000E30B600BC230A128A111030831652
:100C9000B6004708B700992311308316B600210823
:100CA0000139B700992312308316B6002D08B7001A
:100CB00099230A128A1548250A128A11812E831651
:100CC00023080319592E013A0319E12B033A03199A
:100CD0001C2C013A0319572C073A0319A62C013A88
:100CE0000319002D033A03193A2D013A0319702D07
:100CF0000F3A0319892D013A0319AC2D033A031950
:100D0000D62D8312080083120313C300903A031DEB
:100D10008D2E0430C1001030982EB0304306031DD4
:100D2000952E0530C1001D30982E0630C1002A30A6
:100D3000C2008316AE0183124308183E8400831755
:100D4000831600182E1483124208053E8400831770
:100D50008316801AAE1483124308183E840083174A
:100D6000831680182E1583124308183E84008317BB
:100D700083160019AE15831241088316B6002E089B
:100D8000B700992B83160313AE0120182E14A01957
:100D9000AE14201A2E151330B6002E08B700992B6A
:100DA000F601F401F50172087304031900341F30D1
:100DB000F6040310F60AF20DF30D031CDA2EF30C01
:100DC000F20C73087102031DE72E72087002031CF7
:100DD000EF2E7208F0027308031C730AF102F40D7F
:100DE000F50DF60BF61ADF2EF61FFB2EF409F40AAA
:100DF0000319F503F5097408F2007508F300761F6E
:100E00000034F009F00A0319F103F1090034000875
:100E1000F000840A0008F100840A0008F200840A45
:100E20000008F300142F840183120313E301F31F5E
:100E3000282F0310FF30F007F009031CF107F10918
:100E4000031CF207F209031CF307F3096317E31706
:100E500077088039E306F71F3F2F0310FF30F407B0
:100E6000F409031CF507F509031CF607F609031C32
:100E7000F707F7093F2F840183120313E301F801F9
:100E8000F901FA01FB01740875047604770403196B
:100E90004C2FC030E305572FF001F101F201F301AF
:100EA000F12F0310F40DF50DF60DF70DE30AF71F02
:100EB000512FE30A0310F80DF90DFA0DFB0D770819
:100EC0007302031D6D2F76087202031D6D2F7508C6
:100ED0007102031D6D2F74087002031C7F2F78149C
:100EE0007408F0027508031C750FF1027608031CE4
:100EF000760FF2027708031C770FF3020310F70C4A
:100F0000F60CF50CF40CE30363083F39031D5A2F6C
:100F1000631F972F0310FF30F007F009031CF10740
:100F2000F109031CF207F209031CF307F309700827
:100F3000F4007108F5007208F6007308F7007808ED
:100F4000F0007908F1007A08F2007B08F300E31F53
:100F5000F12F0310FF30F007F009031CF107F1092E
:100F6000031CF207F209031CF307F309F12F8401B4
:100F70007008F8007108F9007208FA007308FB00A5
:100F8000F201F301F001F1010310FB0CFA0CF90C72
:100F9000F80C031CD92F7408F00775080318750F97
:100FA000F10776080318760FF20777080318770F12
:100FB000F307780879047A047B040319F12F0310EE
:100FC000F40DF50DF60DF70DC42F0008F000840A9E
:100FD0000008F100840A0008F200840A0008F30007
:100FE000B82F840803190034730880008403720842
:100FF000800084037108800084037008800000343E
:10100000073083120313BA000800831203179515E3
:10101000A215AF159030831603132406031D142860
:101020008312031795111D28B0302406831203176D
:10103000031D1C28A2111D28AF11831603132017AE
:1010400083120800831203133C08053CCD003808C6
:10105000073A03192F283808CD023A08CD07063081
:10106000CC004C084D0203183C28CC034C08323EFF
:1010700084008313800131283A08CC00CC0803197E
:101080005628CC03CD034C08323E8400831300085D
:10109000CB004D08323E840083134B0880003E286D
:1010A000CD034D08323E840083138001CD08031D1B
:1010B00050283208A5003308A7003408A3003508DB
:1010C000A6003608A4000A168A1556250A128A15A3
:1010D0002008CE002108CF002208D000D10107301F
:1010E000BA008316CA1183124E08F0004F08F100AF
:1010F0005008F2005108F300B91C0800F009F1098A
:10110000F209F309F00A0319F10A0319F20A0319A3
:10111000F30A080083120313C60022207008C700D8
:101120007108C8007208C9007308CA004708CB00DC
:101130004808CC004908CD004A08CE0046080A16E7
:101140008A11F5200A128A157008C7007108C800B4
:101150007208C9007308CA004608183E8400831745
:10116000001CCD284708F0004808F1004908F200AB
:101170004A08F300F009F109F209F309F00A03192A
:10118000F10A0319F20A0319F30A7008C70071087B
:10119000C8007208C9007308CA004608183E8400D7
:1011A0008317001DD8284A0DCA0CC90CC80CC70CDF
:1011B0004708F0004808F1004908F2004A08F30027
:1011C0000800831203173F08F0004008F1004108AF
:1011D000F2004208F300F009F109F209F309F00AFC
:1011E0000319F10A0319F20A0319F30A7008BF0080
:1011F0007108C0007208C1007308C2000313080020
:1012000083120313BD000317C11F0829FF30C20456
:1012100003133D08183E84008317001C1029E120A9
:101220003D080C3E840083170008F000840A000883
:10123000F100840A0008F200840A0008F300700834
:101240000317BF077108031C2A29710A0319F20A40
:101250000319F30AC0077208031C3129720A031923
:10126000F30AC10773080318730AC20703133D0882
:10127000173E84008317800803191E2A3D08840046
:1012800083170008F000840A0008F100840A0008AF
:10129000F200840A0008F300700803173F02F4000C
:1012A0004008F5007108031C710FF5024108F600B3
:1012B0007208031C720FF6024208F7007308031C41
:1012C000730FF70274080313CC007508CD0076087D
:1012D000CE007708CF000A128A1171230A128A15EC
:1012E0007008BE007108BF007208C0007308C1001A
:1012F0003D08173E840083170008F000F101F20159
:10130000F3017308803AF4004108803A7402031D27
:10131000932940087202031D93293F087102031D9F
:1013200093293E087002831203133D080318A8296D
:10133000143E8400831780013D08103E840083170B
:101340008001840A8001840A8001840A80011E2AA7
:10135000143E84008317083000023D080318082A51
:10136000143E84008317800A3D08103E84008317D2
:101370000008F000840A0008F100840A0008F20066
:10138000840A0008F30003173F087007F40071088F
:10139000F50040080318400FF5077208F6004108F1
:1013A0000318410FF6077308F70042080318420FAD
:1013B000F70774080313BE007508BF007608C00065
:1013C0007708C1003D08103E840083173E08800066
:1013D000840A3F088000840A40088000840A41088B
:1013E00080003D08143E840083170008083A031D5E
:1013F0001E2A3E08F0003F08F1004008F2004108B4
:10140000F30003300A168A1551240A128A15152A88
:10141000840083170008F000840A0008F100840AA1
:101420000008F200840A0008F30070080317BF00E8
:101430007108C0007208C1007308C20003133D08A0
:101440008400831703173F088000840A4008800047
:10145000840A41088000840A42088000831603132E
:10146000A01C362A83123D08083E392A83123D0803
:10147000043E840083170008F000840A0008F1008D
:10148000840A0008F200840A0008F30070080317B9
:10149000BF0271080318512A710A0319F20A0319CD
:1014A000F30AC00272080318582A720A0319F30AD1
:1014B000C1027308031C730AC20203133D08183EDD
:1014C00084008317801C652AE1203D08183E8400B3
:1014D0008317001D712A03100317BF0DC00DC10D26
:1014E000C20D0313080083120313BD00093E8400DC
:1014F00083170008F000840A0008F100840A00083D
:10150000F200840A0008F3007008BE007108BF00F2
:101510007208C0007308C1003D0884008317000BE7
:10152000A92A4008C2000F30C005C1013E080317B8
:10153000BF0003133F080317C0000313400803173D
:10154000C100031341080317C2000313421E080021
:10155000DF2A3D08840083170008023A031DE12AB0
:101560004108C20040080F39A5003F0E0F39A700FF
:101570003F080F39A3003E0E0F39A6003E080F3971
:10158000A4000A168A1556250A128A152008BE00DC
:101590002108BF002208C000C1013E080317BF0098
:1015A00003133F080317C000031340080317C100CB
:1015B000031341080317C2000313421C0800E12073
:1015C000F12AC1013E080317BF0003133F080317A8
:1015D000C000031340080317C10003134108031799
:1015E000C200031308008B13831603132B08A900F2
:1015F0002C08AA00A0128B17831208003C30F200BE
:101600000230F300831603132D08F000F1010A16CF
:101610008A15FE240A128A157408AB007508AC00FE
:10162000F32A83160313A608031D202B03179C011E
:101630009D019E019F01BC01BD01BE01BF01792B2F
:101640002608B600B6030310B60D0310B60D03103E
:10165000B60D2C30B6073608D32383162E082F0874
:10166000300831082E088312CB0083162F0883120E
:10167000CC00831630088312CD0083163108831204
:10168000CE0090300A168A11F5200A128A157008C9
:10169000831603179C0071089D0072089E00730852
:1016A0009F000313360AB600D32383162E082F0893
:1016B000300831082E088312CB0083162F088312BE
:1016C000CC00831630088312CD00831631088312B4
:1016D000CE00B0300A168A11F5200A128A15700859
:1016E00083160317BC007108BD007208BE007308A2
:1016F000BF00031383120800AB2B0A128A1548257A
:101700000A128A15B62B1E308312C1004630C20061
:1017100090300A168A1546274B30C1004630C20069
:10172000B0300A168A1546276B30C1004630C20019
:10173000D0300A168A1546270A128A15B62B1123AD
:1017400014308316B6002608B7000A128A119923AE
:101750000A128A157D2B83160313230803197D2B88
:10176000013A0319832B033A03199F2B83120800B4
:10177000831603133608831203178D0083168C1308
:101780000C1483120C0883160313B700831208008D
:10179000B82383163708AE00B60AB8238316370875
:1017A000AF0083120800B82383163708AE00B60ACC
:1017B000B82383163708AF00B60AB8238316370854
:1017C000B000B60AB82383163708B10083120800A8
:1017D00083160313B601B82383163708853A031D11
:1017E000EA2CB601B60AB823831637080317A700F8
:1017F00004300313B600B82383163708AE0003176E
:10180000281003132E1C062C031728148312031709
:10181000951283160313AE1C112C83120317951611
:1018200083160317A81003132E1D182C0317A814D2
:10183000031728110313AE1D1F2C031728150230A0
:101840000313B600B823831637080317C700053003
:101850000313B600B82383163708AE0003174810E9
:1018600003132E1C352C0317481483120317A212DE
:1018700083160313AE1C402C83120317A216831683
:101880000317C81003132E1D472C0317C814031782
:1018900048110313AE1D4E2C0317481503300313D4
:1018A000B600B823831637080317E7000630031382
:1018B000B600B82383163708AE0003176810031369
:1018C0002E1C642C0317681483120317AF1283169F
:1018D0000313AE1C6F2C83120317AF168316031766
:1018E000E81003132E1D762C0317E8140317681154
:1018F0000313AE1D7D2C0317681507300313B600C4
:10190000B8238316370883120317900010300A1685
:101910008A11F0230A128A1508308316B600B823FC
:1019200083163708831203179D001D300A168A118B
:10193000F0230A128A1509308316B600B8238316DD
:10194000370883120317AA002A300A168A11F023D7
:101950000A128A150A308316B600C8230A128A159D
:1019600083162E080317A50003132F080317A600DC
:101970000C300313B600C8230A128A1583162E08EA
:101980000317C50003132F080317C6000E300313F7
:10199000B600C8230A128A1583162E080317E5001D
:1019A00003132F080317E60010300313B600B82303
:1019B00083163708C7001130B600B82383162108F4
:1019C0003706FE393706A1001230B600B823831659
:1019D0003708AD001730B600D3230A128A158316D4
:1019E0002E080317940003132F0803179500031301
:1019F00030080317960003133108031797001B30B4
:101A00000313B600D3230A128A1583162E08031770
:101A1000B40003132F080317B5000313300803178E
:101A2000B600031331080317B7001F300313B600C5
:101A3000D3230A128A1583162E080317D400031322
:101A40002F080317D500031330080317D60003131C
:101A500031080317D70013300313B600B8238316D9
:101A60003708AE002E1C362D2014CA14AE18A0154F
:101A70002E1920161430B600B82383163708AE008E
:101A8000A60011230A128A1596308316A700FE2A93
:101A900083160317AF080319562D90300A168A15BE
:101AA000D4240A128A1583160317AF01CF0803192D
:101AB000622DB0300A168A15D4240A128A158316AC
:101AC0000317CF01EF0803196E2DD0300A168A15BF
:101AD000D4240A128A1583160317EF01E330031387
:101AE000CA0507308312BA008316A20183120800C8
:101AF000831603132208023A031D882D24080A16B0
:101B00008A11D8220A128A1548250A128A15CD2D63
:101B10002208033A031D932D24080A168A15F62677
:101B20000A128A15842D2208053A031DB82D831246
:101B30003A08073A83160319B12D2308043A031D06
:101B4000A72D0A168A15AF250A128A15B22D230869
:101B5000053A031DB22D0A168A1529250A128A157F
:101B6000B22DA30A0A128A11DA230A128A15CD2D80
:101B70002208073A031DC32DA30A0A168A118824D6
:101B80000A128A15CD2D2208083A031DCD2DA30A6D
:101B90000A128A157C230A128A15831208008312FE
:101BA00003133A08073A031DDF2D83162208053A6E
:101BB000031DDE2DA3030A128A11DA2B492D3A08E0
:101BC0003806031DEA2D0730B800831624080A16CC
:101BD0008A118328BA08031DEE2D482DBA038316F7
:101BE00024080A168A11832883120313AF08031DE1
:101BF000FB2D9030022E2F08023A031D012EB0302B
:101C0000022ED030BD0083162208023A031D122E88
:101C1000240883123D06031D112E3A08073A0319C2
:101C2000182E8316A208031D292EA01C222E831213
:101C30003D080A168A11D8220A128A1548250A1266
:101C40008A15292E0230A2004A1583123D088316F8
:101C5000A4008312080083160313A208031D3A2E62
:101C60000130A0060230CA060A128A11C2260A12E0
:101C70008A15432E2208043A031D432E8030A00605
:101C800048250A128A158312080083120313C40020
:101C90000A168A15D424BA01B9100730B8004108D1
:101CA000BB004208BC003911C308031D39154408A4
:101CB0001F3E840083178001800A8316CA15831291
:101CC00044088316A400831244080A168A11832844
:101CD000831203132F08043A031D702EBE01782EC1
:101CE0002F08033CBE0003103E0DBE072E03BE07A7
:101CF00083162208023A8312031D972E3A08073AE8
:101D0000031D972E8316201C8A2E03308312C100D8
:101D100002308E2E02308312C1000330C200C30194
:101D2000C30A8316240845260A128A1583123A0824
:101D3000073A0319BF2E3808073A031DAA2E3B089D
:101D40003A0203180800BA08031DB02EBE08031992
:101D50000800B02E3C083807BD003A0203180800FE
:101D6000BA0A3A03323E840083133E088000831689
:101D700024080A168A1183200A128A15452F831611
:101D80002208043A0319142F2B2F05308316A200C2
:101D9000A301A30A0A128A11DA230A128A15452F0F
:101DA00006308316A2004B308312C1000330C200FC
:101DB00090300A168A1546274430C1000330C2000D
:101DC000B0300A168A154627D0300A168A15D42450
:101DD0000A128A15452F07308316A200A301A30A11
:101DE0000A168A1188240A128A15452F083083168C
:101DF000A200A3013F2F8316211C062F0830A00646
:101E000020120A128A11C2260A128A1548250A12BD
:101E10008A15452F8316211C062F1030A006A0110D
:101E2000012F8316A016062F83123E080319C52E14
:101E3000023A0319D02E073A0319EB2E033A03197D
:101E4000F62E013A0319FB2E0F3A03190A2F013A15
:101E50000319112F062F2208073A031D372F83126B
:101E6000BE08031908003E088316A600EF2E2208BC
:101E7000083A8312031D08003E088316A600A30A31
:101E80000A128A157C230A128A1583120800831607
:101E900003132208023A8312031D672F3A08073AF8
:101EA000031D672F8316201C5A2F03308312C10095
:101EB00002305E2F02308312C1000330C200C30122
:101EC000C30A8316240845260A128A1583123A0883
:101ED000073A031D391D08000230B906831624088D
:101EE0000A168A118328831603132208023A8312E2
:101EF000031D932F3A08073A031D932F8316201CC6
:101F0000862F03308312C10002308A2F02308312E1
:101F1000C1000330C200C301C30A8316240845264A
:101F20000A128A1583123A08073A0319080038087A
:101F3000073A031D0800BC08031908003A08B80056
:101F4000831624080A168A11832883120313AF0804
:101F5000031DAF2F90308316A4001030B72F2F0829
:101F6000023A031DB92FB0308316A4001D30A5001E
:101F7000F22FD0308316A4002A30B72F0330A200EE
:101F8000201CCF2F03308312C1000230C200C301D6
:101F9000C30A8316240845260A128A15FE2F02302A
:101FA0008312C1000330C62F0A128A1505200A12B7
:101FB0008A1548250A128A15FE2F0A168A11DD2174
:101FC0000A128A11DA230A128A15FE2F24080A1629
:101FD0008A153E24831624080A128A1183260A12BF
:101FE0008A15D92F22080319BE2F043A0319D42FBA
:101FF000013A0319DD2F033A0319E62F8312080073
:1020000082073F3406345B344F3466346D347D349C
:1020100007347F346F3477347C3439345E34793428
:02202000713419
:1020240083120317170B2F289730180203181B2845
:10203400980A10300A128A15732290300A128A15EF
:10204400002190300A168A11C5260A168A11031730
:1020540012089600023097001512240B4A28973074
:10206400250203183628A50A1D300A128A15732280
:10207400B0300A128A150021B0300A168A11C5261A
:102084000A168A1103171F08A3000230A4002212A3
:10209400310B6C289730320203185128B20A2A30C7
:1020A4000A128A157322D0300A128A1500210A16E0
:1020B4008A118316A01D201A6528D0300A168A11A9
:1020C400C5260A168A11831203172C08B0000230A1
:1020D400B1002F121708023A03197228151E81281D
:1020E4002408023A03197828221E81283108023A6A
:1020F40003197E282F1E81289701A401B10103131F
:10210400080083120313C8001F3E84008317000BCA
:102114000800BA08031D9A284808193E840083174A
:102124000A168A1101200A168A118000C901BE28E4
:102134003A08C700C9013A0849060319BF28C7036A
:102144004708323E840083130008C50010308A001B
:10215400450800200A168A11C60049084807193E96
:102164008400831746088000C90A9D284908480747
:10217400193E840083178001C90A06304902031CF2
:10218400B8283808073A0319DE2838083A02C90083
:10219400B808031DD82849084807193E8400831746
:1021A4000A168A1101200A168A1180004908480774
:1021B400193E840083178017B91C0800B808031D52
:1021C400BA08031DED283A0848071A3E840083170D
:1021D4004030800008003A084807193E84008317FD
:1021E40040308000080083120313CF004B08F40032
:1021F4004C08F5004D08F6004E08F7004F08153E50
:10220400840083170008F000840A0008F100F2013A
:10221400F3010A128A11B7270A168A117008D0002E
:102224007108D1007208D2007308D3003230D40090
:10223400D31F1E29D409D40A5408D0070130031827
:10224400D1070318D2070318D3076430F400F5014B
:10225400F601F7015030840083130A128A1107270C
:102264000A168A1183160313201C5C293230F400E9
:10227400F501F601F70183125030840083130A122A
:102284008A11E527193083120313D007013003188C
:10229400D1070318D2070318D3077F30F400F501E0
:1022A400F601F7015030840083130A128A110727BC
:1022B4000A168A11831203135008F0005108F10022
:1022C4005208F2005308F300080038308312031355
:1022D4008500831685010130831286007E308316C3
:1022E400860083128701043083168700D43081006E
:1022F400313083129000063092009430831692009D
:1023040007308C0068308B0006309F000430831245
:1023140097000800672110300A168A1176241D30B0
:102324000A168A1176242A300A168A117624103065
:10233400BD0090300A168A153F251D30BD00B0300F
:102344000A168A153F252A30BD00D0300A168A1590
:102354003F250A168A1538240A128A1500200A1203
:102364008A15E823FE30C1000230C20090300A16FC
:102374008A154627F830C1000230C200B0300A1670
:102384008A154627F230C1000230C200D0300A1646
:102394008A1546278316A201A20A8B170A168A11E8
:1023A40012200A168A1160230A168A11D1250A16E8
:1023B4008A116400D029372A2408183E8400831720
:1023C40001308006532A2408183E84008317023003
:1023D400E329250884008317800A250884008317CD
:1023E4000008033A031DFA29250884008317800195
:0C23F40025080A168A11F0230A168A1127
:10240000532A05308312C100C201C3018316240878
:102410000A128A1545260A168A11532A0230022A00
:102420002508053E840083172030E329C70B532A73
:102430000530C700532A0130A106532AAD08031DF9
:10244000232A0F302E2A2D080F3A031D292A1E3069
:102450002E2A2D081E3A031D302A3C30AD00312AA9
:10246000AD010A128A15FE220A168A11532A831612
:1024700003132308F0000130F002031C532A093033
:1024800070020318532A12308A004A30700703186A
:102490008A0A8200DE29E529EB29012A0E2A102A60
:1024A000162A1B2A1E2A8312080083120313D00047
:1024B0002030F4000330F500F601F7014C08F0007D
:1024C0004D08F1004E08F2004F08F3000A128A117D
:1024D000B7270A168A117008D1007108D200720855
:1024E000D3007308D4005008153E840083170008F9
:1024F000F000840A0008F1000310F10CF00C7008E1
:10250000D500D41F852AD509D50A5508D107013031
:102510000318D2070318D3070318D4075008153E31
:10252000840083170008F000840A0008F100700896
:10253000F4007108F500F601F701513084008313AF
:102540000A128A1107270A168A1183160313201C00
:10255000CD2A7F30F400F501F601F70183125130E6
:10256000840083130A128A11E5271930831203139A
:10257000D10701300318D2070318D3070318D40773
:102580003230F400F501F601F70151308400831375
:102590000A128A1107270A168A1183120313510897
:1025A000F0005208F1005308F2005408F30008004C
:1025B00083120313C1003A08073A031D1D2B41087B
:1025C000840083170008F000840A0008F100840AE0
:1025D0000008F200840A0008F3007008C2007108C5
:1025E000C3007208C4007308C5008316A01C092B21
:1025F00083124108083E8400831742088000840A41
:1026000043088000840A44088000840A450880004A
:10261000080083124108043E8400831742088000AA
:10262000840A43088000840A44088000840A45081C
:10263000800041080A168A15802D41080A128A1561
:102640008A200A168A117008C2007108C300720835
:10265000C4007308C5004108043E840083170008C5
:10266000F000840A0008F100840A0008F200840ADD
:102670000008F3007008C2077108031C442B710A9C
:102680000319F20A0319F30AC3077208031C4B2B40
:10269000720A0319F30AC40773080318730AC507FB
:1026A0004108043E8400831742088000840A4308DE
:1026B0008000840A44088000840A450880000800DD
:1026C00083120313391C0800A808031D912BAE01C7
:1026D00005302E022E080318852B293E8400831313
:1026E0000008B100AF01B119842BAF0A311A842B55
:1026F000AF0AB11A842BAF0A311B842BAF0AB11B6E
:10270000842BAF0AAE0A682B2E08053A0319EE2B6C
:102710002F08053A0319EE2BB001B00AA801A80A48
:10272000EE2B2E08293E840083130008B100AF0869
:10273000031D9C2B0830AD2B2F0BA02B1030AD2B85
:102740002F08023A031DA62B2030AD2B2F08033A89
:10275000031DAC2B4030AD2B8030B105B108031DFB
:10276000B52BB00BEE2BA801EE2B280BE52BB00AF6
:102770003008053A031DEE2B8316A01EC52B0A1246
:102780008A15F3220A168A11E22B0530F100831212
:102790002E080A168A1572242F07F0007007F00021
:1027A0001830DC007008013E0A128A11C122F000C4
:1027B0000A128A11C222DC0070080A128A11C12290
:1027C0000A168A110230A800EE2B2808023A031DCF
:1027D000EE2B3008053A0319EE2BB00A3910080029
:1027E00083120313BE0084008317000B1D2C3E0AC6
:1027F00084008317183080003E08053E840083174C
:1028000000103E08053E8400831780103E08033EFA
:1028100084008317FA3080003E08053E8400831749
:1028200000153E08053E8400831780153E08023ED1
:10283000840083179930800008003E0884008317C5
:102840000008023A031D4A2C3E0A840083171C30FC
:1028500080003E08053E8400831700143E08053EB4
:102860008400831780103E08033E840083171F30C6
:1028700080003E08053E8400831700113E08053E97
:102880008400831780113E08023E840083171F30A6
:10289000800008003E0A84008317183080003E083C
:1028A000053E8400831700143E08053E840083170C
:1028B00080143E08033E840083171F3080003E08CA
:1028C000043E840083173E3080003E08053E8400AD
:1028D000831700113E08053E8400831780113E08CF
:1028E000023E840083171F30800008008312031308
:1028F000BD00073E8400831780013D08053E84002B
:10290000831780163D088400831780013D08F02B53
:10291000192D1E308312C1004630C20090300A16B5
:102920008A1546274B30C1004630C200B0300A1627
:102930008A1546276730C1004630C200D0300A16DB
:102940008A1546270A168A112A2D80308312C10063
:102950004630C20090300A168A154627D0300A1633
:102960008A15D4240A168A118316201CDE2C033003
:102970008312C1000230C200C301B0300A128A15AE
:1029800045260A168A112A2D0A128A152220700855
:102990008316AE007108AF007208B0007308B10072
:1029A00079308312C1004630C20090300A168A1571
:1029B00046270A168A1183162018B72C0230831274
:1029C000C1000330BB2CA6080319132D0A128A1567
:1029D000222070088316B2007108B3007208B40098
:1029E0007308B5002608B600B6030310B60D031031
:1029F000B60D0310B60D2C30B6072E082F08300880
:102A0000310836080A128A11C62383163208AE002E
:102A10003308AF003408B0003508B100360AB600FC
:102A20000A128A11C6230A128A1548250A168A1123
:102A30002A2D8316031323080319132D013A0319B2
:102A4000892C033A0319A52C013A0319C42C073A1F
:102A50000319E32C8312080083120B1D472D031763
:102A60001708023A031D372D960B372D97012408BE
:102A7000023A031D3E2DA30B3E2DA4013108023A5C
:102A8000031D452DB00B452DB1010B11831203130E
:102A90000C1C8B2D8316B90A0319BA0AA70803194F
:102AA000632DA70B632D0730C9000A168A15E92488
:102AB0000A168A157E240A168A1526260A168A11EF
:102AC0000A308316A8002A08290403196F2DFF3045
:102AD000A907031CAA032A0829040319A016A80899
:102AE0000319862DA80B862D831203179808031946
:102AF0001516A50803192216B20803192F169801F6
:102B0000A501B2010A3083160313A800B808031DFB
:102B1000B80383120C108C1C08008316C80A4708DF
:102B20004802031C982D0A168A155C240A168A117D
:102B3000053083164802031CCE2D07304902031CC2
:102B4000AE2D83123918AC2D0A168A15E9240A16FF
:102B50008A15AC260A168A118316C901A01ACC2D33
:102B60000A168A15E9240A168A11063083164902C4
:102B70000318C62D0A168A15B0240A168A159F2432
:102B80000A168A158E240A168A11CB2D0A168A1562
:102B900013250A168A118316C801C90A83128C10DC
:102BA000080083160313211CC32E2208023A031DBA
:102BB000E72D83123A08073A83160319201DE72DE3
:102BC0000A128A1578250A168A1183162011A0196F
:102BD000EB2D201EC32EB808031DC32E0A30B800EB
:102BE000C301C401C501C601201DBE2E3F083B0222
:102BF000F0003C08F1004008031C400FF1023D08C2
:102C0000F2004108031C410FF2023E08F3004208A3
:102C1000031C420FF30270088312CC007108CD0030
:102C20007208CE007308CF000A128A11712370084F
:102C3000BD007108BE007208BF007308C0003D08E7
:102C4000F4003E08F5003F08F6004008F700603049
:102C5000F0003430F1003C30F2000230F3000A1290
:102C60008A1113270A168A1170088316C300710887
:102C7000C4007208C5007308C600201EBC2E0317CE
:102C800014081002F0001108F1001508031C150FBC
:102C9000F1021208F2001608031C160FF2021308C4
:102CA000F3001708031C170FF302700883120313B5
:102CB000BD007108BE007208BF007308C000C01FCD
:102CC000652EBD01BE01BF01C0016430F400F501F5
:102CD000F601F7013D30840083130A128A11E527BB
:102CE000831603172508F4002608F500F601F701FE
:102CF000831203133D30840083130A128A110727BD
:102D00007030F400F530F500F601F701831203137B
:102D10003D30840083130A128A11E527E030F40065
:102D20002E30F500F601F701831203133D308400C5
:102D300083130A128A110727831203133D08F40034
:102D40003E08F5003F08F6004008F7008316C33040
:102D5000840083130A128A11E5271030F40027300B
:102D6000F500F601F70183160313C33084008313C3
:102D70000A128A1107278316031320110A168A15CF
:102D8000A0270A168A118312080083120313BD00BC
:102D90001F3E840083178008031D08008316A01FB0
:102DA0001F2F831203173F080313C20003174008A5
:102DB0000313C300031741080313C4000317420899
:102DC0000313C5003D08193E8400831710308A00A4
:102DD00042080F39002080003D081A3E8400831706
:102DE00010308A00420E0F39002080003D081B3E43
:102DF0008400831710308A0043080F3900208000B8
:102E00003D081C3E8400831710308A00430E0F39A2
:102E1000002080003D081D3E8400831710308A008A
:102E200044080F39002080003D081E3E84008317AF
:102E300010308A00440E0F390020800008008312F1
:102E400003173F080313CC00031740080313CD00FA
:102E5000031741080313CE00031742080313CF00E2
:102E60000A128A1171237008BE007108BF0072082F
:102E7000C0007308C1003E08CC003F08CD004008E8
:102E8000CE004108CF003D080A168A1155220A16C5
:102E90008A117008BE007108BF007208C000730874
:102EA000C1003E08C2003F08C3004008C4004108FA
:102EB000C5000330F000450DC50CC40CC30CC20C9A
:102EC000F00B5B2F4208A0004308A1004408A200B9
:102ED0000A168A15E6250A168A110A302502031CED
:102EE0007E2F4030C6005C30C7003830C8007130DB
:102EF000C9005C30CA004030CB00DB2F10308A00A4
:102F000024080020C60010308A0026080020C700D0
:102F100010308A00230800200A168A11C800C9014F
:102F2000CA01CB0183162018992F83123E1D9A2FB8
:102F3000C6178312A508031DBA2F8316201CAB2FBA
:102F40008312A708031DAB2F0317C21FCC2F4030DD
:102F50000313C900CC2F10308A00831227080020E9
:102F60000A168A11C9000317C21FCC2F4030031361
:102F7000CA00CC2F10308A0027080020C90010306A
:102F80008A00250800200A168A11CA000317C21FEA
:102F9000CC2F40300313CB0083160313201CD32FF8
:102FA0008312C817D52F8312C9173D08183E840015
:102FB00083170019CB173D08193E84008317460874
:102FC00080003D081A3E84008317470880003D08B2
:102FD0001B3E84008317480880003D081C3E840087
:102FE0008317490880003D081D3E840083174A0866
:102FF00080003D081E3E840083174B0880000800B7
:1030000082074F340334523403344F340334523480
:1030100003344F34033455340334583403345534B3
:1030200003345B340334553403345E340334613485
:103030000334613403346134033464340334673457
:103040000334613403346134033461340334613450
:1030500003346A3403346134033461340334613437
:1030600003346D340334820777347C3439345E346E
:10307000793471343D34743404341E3400343834BB
:10308000003454345C347334003450346D34783448
:0C3090003E341C34003400346E345B34D9
:10386A00031383120800053083160313C70083125B
:10387A00080083120313BD00183E84008317043026
:10388A008006080083160313A208031D4F2C043078
:10389A00A2004A1683120800F400F40AF40303197A
:1038AA000034730DF30CF20CF10CF00C532C831250
:1038BA000313051087018514051586178510051150
:1038CA008613080083160313A208031D702C023006
:1038DA00A0060130CA0683120800F00000307118F1
:1038EA0070070310F00D0310F10CF108031908001A
:1038FA00742C973083120317180203189515973002
:10390A0025020318A215973032020318AF150313C4
:10391A000800831603134908E93E84008317000848
:10392A008312D600051056190514870086178617C4
:10393A0086130800831603134908C93E84008317B7
:10394A0000088312D60005105619051487000515BC
:10395A00051505110800831603134908A93E8400BA
:10396A00831700088312D60005105619051487001C
:10397A00851485148510080083120313D700D02CF0
:10398A000103D600560801060319CD2C6400C72C82
:10399A00D70383120313D70803190800C52C83120F
:1039AA000313C5001F3E8400831702308000C6013E
:1039BA0046084507193E840083178001C60A063067
:1039CA00460203180800DD2C8316031349088312E4
:1039DA00D600561CF22C8515F32C8511D61CF72C13
:1039EA000516F82C0512561DFC2C851608008512A2
:1039FA000800F401F5010310F30CF20C031C0C2D62
:103A0A007008F40771080318710AF5070310F00D1E
:103A1A00F10D7208730403190034002D8312031385
:103A2A008701051083164A088312D6005618071410
:103A3A00D618871456190514D6198715561A071653
:103A4A0085148514851008000A128A1522200A1680
:103A5A008A1570088316AE007108AF007208B000AC
:103A6A007308B1002408173E840083172E088000CB
:103A7A008312080083120313BE001F3E84008317BB
:103A8A00023080003E08173E840083170C30800005
:103A9A003E08153E840083178001840A083080009E
:103AAA00080083120313A20126082707A000A00713
:103ABA00250DA100230E2307A0072708A107A00DA3
:103ACA00A10D230E2607A007250E03180138A1070A
:103ADA00270EA002031CA1030310A00DA10D0318B9
:103AEA002214250E2407A007250803182503A1027E
:103AFA0003138312080083120313C600903A031DAE
:103B0A00882D17308F2DB0304606031D8E2D1B30A1
:103B1A008F2D1F30C7004608043E84008317000813
:103B2A00F000840A0008F100840A0008F200840AFE
:103B3A000008F30070088316AE007108AF0072081F
:103B4A00B0007308B100831247088316B6000A1240
:103B5A008A11C72B0A128A1522200A168A1570089A
:103B6A008316AE007108AF007208B0007308B10086
:103B7A003004031DE42D0A30F200F3012E08F00090
:103B8A002F08F1000A128A11D0260A168A1574081B
:103B9A00AE007508AF0009302F02C53003192E0296
:103BAA000318E42D2F082E040319E42D2408153ECA
:103BBA00840083172E088000840A2F08800083124D
:103BCA00080083120313210E0F39DC3EA700A70752
:103BDA00983EA300903EA40021080F39A307A3072B
:103BEA00A407DF3EA600A607A607200E0F39A607E0
:063BFA00A407A60DA40DB6
:103C0000A409A40D20080F39A407A70D1030A500A2
:103C1000221C122E0430A402A6070530A307A70712
:103C20000630A5070A30A407A603031C132EA60717
:103C3000A303031C172EA307A703031C1B2EA70710
:103C4000A503031C1F2E0313831208008312031302
:103C50008701051003179519302E031387140317D6
:103C6000A219352E031387150317AF19392E031325
:103C7000871603130610F4300A168A15C124061499
:103C8000871087118712F4300A168A15C1240A1684
:103C90008A1507100510071203179519522E0313E2
:103CA00007140317A219572E031305140317AF198E
:103CB0005B2E0313071603130610F4300A168A1539
:103CC000C1240A168A1506140710051007120800E9
:103CD00083120313C3001F3E840083170230800049
:103CE0004108C7004208C8004708A0004808A100D2
:103CF000A2010A168A15E6250A168A152508CD009E
:103D00002708CC002308CB002608CA002408C900D5
:103D10000430C6004608493E840083138008031D12
:103D2000932EC60B8A2EC50145084602031C0800C7
:103D30004508493E840083130008C4004508430732
:103D4000193E8400831710308A00440800200A16A8
:103D50008A158000C50A942E831203138701F83058
:103D60008316870483128514051107108710051028
:103D70000430D7000708D600D70BBA2E0708A900D1
:103D8000851005150430D7000708D600D70BC42EC0
:103D90000708AA00051107140430D7000708D60049
:103DA000D70BCE2E0708AB00071087140430D700BE
:103DB0000708D600D70BD82E0708AC0087100514CB
:103DC0000430D7000708D600D70BE22E0708AD0055
:103DD00007308316870583120510870185140515A2
:103DE00086178510051186133914080083120313F2
:103DF000C1000A128A158A200A168A157008C200A4
:103E00007108C3007208C4007308C5008316A01CA3
:103E10000C2F831241080F2F83124108043E8400A7
:103E200083170008F000840A0008F100840A0008E3
:103E3000F200840A0008F3007008C2077108031C2E
:103E4000262F710A0319F20A0319F30AC30772082D
:103E5000031C2D2F720A0319F30AC40773080318F1
:103E6000730AC5074108083E840083174208800092
:103E7000840A43088000840A44088000840A4508B4
:103E800080008316A0144A148312080083120313BF
:103E9000C3001F3E84008317023080000630C70035
:103EA000C801C70348084107DB004208DC005B0883
:103EB0000318DC0A0A128A11C1220A168A15C600E2
:103EC000C60803199B2F4608203A031D692FC50118
:103ED000862F46082D3A031D6F2F4030852F613005
:103EE00046024608031C7D2F9F3EC40018308A00FE
:103EF000440833200A168A15852FD03EC40010309E
:103F00008A00440800200A168A15C500470843079E
:103F1000193E8400831745088000C80A063048020D
:103F200003189B2F512F47084307193E840083171E
:103F30008001C703C80A0630480203180800932FFF
:103F400083160317EF080313031DFE2F4308831284
:103F5000A000831644088312A1008316450883122B
:103F6000A2000A168A15E62510308A0024080020CF
:103F7000C10010308A0026080020C20010308A00DC
:103F800023080020C30010308A0027080020C40046
:103F900010308A00250800200A168A15C500C601BF
:103FA000A508031DE02FC501A708031DE02FC401CC
:103FB000A308031DE02FC301A608031DE02FC201C3
:103FC000410883160317E90083120313420883167E
:103FD0000317EA0083120313430883160317EB0049
:103FE00083120313440883160317EC008312031390
:103FF000450883160317ED00EE0103138312080032
:02400E0076FF3B
:1042000000000000000000000000000000000000AE
:10421000000000000000000000000000000000009E
:10422000000000000000000000000000000000008E
:10423000000000000000000000000000000000007E
:10424000000000000000000000000000000000006E
:10425000000000000000000000000000000000005E
:10426000000000000000000000000000000000004E
:10427000000000000000000000000000000000003E
:10428000000000000000000000000000000000002E
:10429000000000000000000000000000000000001E
:1042A000000000000000000000000000000000000E
:1042B00000000000000000000000000000000000FE
:1042C00000000000000000000000000000000000EE
:1042D00000000000000000000000000000000000DE
:1042E00000000000000000000000000000000000CE
:1042F00000000000000000000000000000000000BE
:1043000000000000000000000000000000000000AD
:10431000000000000000000000000000000000009D
:10432000000000000000000000000000000000008D
:10433000000000000000000000000000000000007D
:10434000000000000000000000000000000000006D
:10435000000000000000000000000000000000005D
:10436000000000000000000000000000000000004D
:10437000000000000000000000000000000000003D
:10438000000000000000000000000000000000002D
:10439000000000000000000000000000000000001D
:1043A000000000000000000000000000000000000D
:1043B00000000000000000000000000000000000FD
:1043C00000000000000000000000000000000000ED
:1043D00000000000000000000000000000000000DD
:1043E00000000000000000000000000000000000CD
:1043F00000000000000000000000000000000000BD
:00000001FF
